:020000040000FA
:10000000B2019E28B216B21EB21232190C28FE3965
:10001000B300321503109928321A1428A60032169C
:100020002B20031819282608322003181928B21E7D
:1000300099282420492032113212B2113608840046
:100040003408841780042A2836088400340980057F
:100050008417800508001E204920242045203308ED
:10006000B2190138A2000830A300A20D03181E2007
:10007000031C242049204520A30B35281E2049209D
:100080003608840034080005FF3E3708840035092F
:1000900027283708840035082128A301A200FF3053
:1000A000A207031CA307031C99280330A100DF301B
:1000B0005B204F28A101E83EA000A109FC30031CF1
:1000C0006428A00703186128A0076400A10F612815
:1000D00020186A28A01C6E2800006E280800A301C2
:1000E000A20002307328A80023082102031D7A28E9
:1000F00022082002043003180130031902302805B9
:10010000031DFF3099281030A800A101A001A70C01
:10011000A60C031C91282208A00723080318230F0C
:10012000A107A10CA00CA50CA40CA80B87282408DF
:100130009928831303138312640008008316FF3089
:100140008600831207309F00831681018312C2301C
:10015000C00064304D200608BE00BF013E08A0006C
:100160003F08A10041086F20031DF3283E08C1008D
:100170000830A600A7013E08A2003F08A300832084
:10018000BE002508BF006400051ECB288030BA00E1
:100190002530BB00CF28E030BA004730BB006400F8
:1001A000051FD528BC01BD01D928FC30BC000E308C
:1001B000BD003A083E07B8003B080318013E3F0760
:1001C000B9000530B6000830B4000530B70004307F
:1001D000B500400804203908042038080420CE3037
:0C01E00004200030022001304D20AB282C
:02400E00383F39
:00000001FF
